:020000020000FC
:100000005BC371C55DC558C357C356C33DC354C315
:1000100053C352C351C350C34FC34EC34DC34CC34C
:1000200058C5475053444F2059542076312E302024
:100030000400436F756E747304004F73632068652A
:1000400061742D757020776169742031356D0400FD
:100050005075736820627574746F6E20746F2070B1
:1000600061737320040057616974696E672E2E2EC8
:10007000040043616C6962726174696F6E2070681C
:100080006173652031200400436F756E74696E677B
:100090002E2E2031732073616D706C6504004361F6
:1000A0006C6962726174696F6E207068617365203B
:1000B0003220040043616C6962726174696F6E2062
:1000C0007068617365203320040043616C6962725B
:1000D0006174696F6E20706861736520342004005C
:1000E000436F756E74696E672E2E363073207361A0
:1000F0006D706C650400436F756E74696E672E2EAB
:100100003130732073616D706C650400436F756EE0
:1001100074696E672E323030732073616D706C6558
:100120000400736C6F77696E672D646F776E2E2E87
:100130002E2004007370656564696E672D75702EDE
:100140002E2E20200400417765736F6D65203A29BB
:1001500020202020202004002020202020202020DB
:1001600020202020202020202020202004004E6F4E
:100170002070756C736520646574656374656420B4
:100180002020040053656C662072756E6E696E6780
:10019000206D6F64652E2E2E0400526573657469A0
:1001A0006E672064656661756C742E2E2E200400C7
:1001B000656570726F6D20636F6E66696720666F2C
:1001C000756E642004004E6F20636F6E6669672051
:1001D000666F756E642C20353025040070776D20B5
:1001E00073657420746F2064656661756C7420207B
:1001F00004005365742070776D20546F3A20307876
:10020000040043616C6962726174696F6E2070688A
:100210006173652035200400436F756E74696E67E5
:100220002E393030732073616D706C650400527527
:100230006E6E696E67206D6F64652E2E2E202020F5
:1002400020200400436F756E74696E672031302082
:1002500042696C6C696F6E20040030313233343582
:100260003637383941424344454603E008B91ED089
:1002700003E008B91BD003E008B918D002E008B9C0
:1002800015D002E008B912D093D008E008B90ED01A
:1002900000E008B90BD00CE008B908D000E008B9BC
:1002A00005D006E008B902D00BD008954598449ACD
:1002B0007FD044980895459A449A74D044980895FC
:1002C00000E008B9F3DF01E008B9F0DF089508E0C5
:1002D00008B9ECDF00E008B9E9DF08950CE008B9DF
:1002E000E5DF00E008B9E2DF089509E008B9DEDFE4
:1002F00004E008B9DBDF08950DE008B9D7DF04E0BA
:1003000008B9D4DF089500E205D00895F1E0E8E5EA
:1003100039D00895102F02950F701F7008B9CBDFE8
:1003200018B9C9DF08950093210113E018B9C3DF9C
:100330000091210110EF0123029508B9BCDF13E001
:1003400018B9B9DF009121011FE0012308B9B3DF1B
:1003500008950093210113E018B9ADDF0091210148
:1003600010EF0123029508B9A6DF0895009321013B
:1003700013E018B9A0DF009121011FE0012308B9A3
:100380009ADF0895C895002D043059F0002D102DE6
:1003900002950F701F7008B98EDF18B98CDF319687
:1003A000F1CF089526EA2A95F1F70000000008959C
:1003B00031E229EC2A95F1F73A95D9F700000000CF
:1003C000089585DFF0E0E2E7DDDF88DFF0E0E8E8D0
:1003D000D9DF08957CDFF0E0EEE9D4DF7FDFF0E0E5
:1003E000E6EFD0DF089573DFF0E0E4EBCBDF76DFFC
:1003F000F0E0E0EEC7DF08956ADFF0E0EAECC2DF8C
:100400006DDFF1E0ECE0BEDF089561DFF2E0E2E0F5
:10041000B9DF64DFF2E0E8E1B5DF089558DFF2E02C
:10042000EEE2B0DF5BDFF2E0E4E4ACDF089564DF2E
:10043000F1E0E2E2A7DF08955FDFF1E0E4E3A2DFAD
:1004400008955ADFF1E0E6E49DDF08950F930295E9
:100450000F70F2E0EAE5E00F08F4F395C895002D7F
:1004600059DF0F910F70F2E0EAE5E00F08F4F39521
:10047000C895002D4FDF08958827579F402C512C99
:10048000469F202C312C569F300C411C581E479FF4
:10049000300C411C581E0895400F511F621F731FDE
:1004A0000895112722273327BB27AA279927881BBE
:1004B000C1E27795679557954795CA9551F020F415
:1004C000800F911FA21FB31FB795A795979587958A
:1004D000F0CF0895002711272227332744275527D7
:1004E0006627772788279927AA27BB27CC27DD27C8
:1004F000EE27FF270895A89572E486ED9BEE9A9566
:10050000F1F78A95D9F77A95C1F773E07A95F1F703
:1005100000000895DD27CC2701E000930201EBDF06
:10052000A89500910201003029F02196CA17DB0737
:10053000B1F708950027009302010895DD27CC2725
:1005400055276627772788279927C8E20ED0000FFE
:10055000111F221F331F441F551F661F771F881F3F
:10056000991FAA1FCA9591F708955F935F70553040
:1005700010F05D5FD52FD52F5F91507F503508F07B
:10058000505D5D0F6F936F70653010F06D5FD62F0B
:10059000D62F6F91607F603508F0605D6D0F7F939F
:1005A0007F70753010F07D5FD72FD72F7F91707FD0
:1005B000703508F0705D7D0F8F938F70853010F06F
:1005C0008D5FD82FD82F8F91807F803508F0805D88
:1005D0008D0F9F939F70953010F09D5FD92FD92F6D
:1005E0009F91907F903508F0905D9D0F0895AF9397
:1005F000AF70A53010F0AD5FDA2FDA2FAF91A07F8A
:10060000A03508F0A05DAD0F0895F999FECF112730
:1006100011BDF1E0EBE2019100BD04E00FBBFA9ADD
:10062000F99AF999FECF139511BD1230A1F7112750
:100630000895F999FECF1127009134010F3F19F465
:1006400002E00093340101BDF1E0E9E0019100BD59
:1006500004E00FBBFA9AF99AF999FECF139511BDF0
:100660001130A1F711270895F999FECF112711BD77
:10067000F1E0EBE2F89AF899FECF00B501931395FB
:1006800011BD1230B9F70895A89501E000932D012E
:1006900017DE1DDEF1E0EEE675DE20DEF1E0E4E8D7
:1006A00071DE01E005BB00E005BD14DF06BD00936F
:1006B00000010093010121C30FEF0DBF02E00EBF47
:1006C00002E0009334010FEF04B907B900270AB91B
:1006D00008B90FEF0BB9C9DDA1DE4B990EC00FEFC2
:1006E00000932B0100932C0190DFEADDF0DDF1E0B7
:1006F000EAE948DEBB27A5E00DDF0FEF0093870096
:100700000FEF0093860002E80093800009E1009358
:100710008100AADF10912C0120912B010FEF1017FF
:100720002007F1F000912B010093890000912C012A
:1007300000938800C5DDCBDDF1E0E0EB23DECEDD0C
:10074000F1E0E2EF1FDE00912B0180DE00912C0131
:100750007DDEBB27A5E0DEDE05E00093030115C0CA
:100760000FE7009389000FEF00938800A9DDAFDD4C
:10077000F1E0E6EC07DEB2DDF1E0ECED03DEBB27F5
:10078000A5E0C8DE01E00093030100E802E00DBB34
:100790000BE00093690001E000936E0000E005BDEE
:1007A000002706BD00930001009301018ED292DE66
:1007B000A89508E10093600006E4009360000091B2
:1007C0000301053041F001E000932E010027009362
:1007D0002F01F7DD92C219DE04E800932E0103E039
:1007E00000932F018AC2EDDD00910901003869F004
:1007F000EAF01DDE30918900209188002D533A40A7
:10080000309389002093880078C21BDEB0E0A5E019
:1008100081DE72DD7BDDDEDD02E0009303010AE0B4
:1008200000932E01002700932F0167C205DEB091CF
:100830008900A09188000DE31AE0A00FB11FB093CA
:100840008900A093880059C2C5DD0AE000932E01FB
:10085000002700932F0100910901003091F00091D1
:1008600009010233F8F0E8DDB0918900A091880019
:1008700006E011E0A00FB11FB0938900A09388009B
:100880003CC2DFDDB0E0A5E045DE36DD3FDDABDDBF
:1008900003E0009303010CE300932E010027009373
:1008A0002F012BC2C4DD3091890020918800265091
:1008B000314030938900209388001FC294DD0CE3FF
:1008C00000932E01002700932F01009109010030B1
:1008D00081F00F37F8F0B0DDB0918900A091880069
:1008E0000BE210E0A00FB11FB0938900A093880025
:1008F00004C2A7DDB0E0A5E00DDE7EDDFDDC06DD97
:1009000004E00093030108EC00932E0100270093FC
:100910002F01F3C18CDD30918900209188002B528A
:1009200030403093890020938800E7C165DD08ECF2
:1009300000932E01002700932F0100910901003040
:1009400081F00F37F8F078DDB0918900A091880030
:100950000CE010E0A00FB11FB0938900A0938800B5
:10096000CCC16FDDB0E0A5E0D5DD4FDDC5DCCEDC70
:1009700005E00093030104E800932E0103E00093D7
:100980002F01BBC154DD30918900209188002C508B
:1009900030403093890020938800AFC136DD49DEB6
:1009A0000091340103950093340104E800932E0173
:1009B00003E000932F0100910901003089F00F3707
:1009C00070F03ADDB0918900A091880003E010E05A
:1009D000A00FB11FB0938900A09388008EC11AC0E8
:1009E00030DD309189002091880030932B012093D5
:1009F0002C010BDEB0E0A5E08DDD10DD7DDC86DCBA
:100A000006E00093030104E800932E0103E0009345
:100A10002F0173C10CDDB0918900A0918800A35013
:100A2000B040B0938900A093880067C1009109018C
:100A300000DE00913401039500933401EFDC08EEF1
:100A400000932E0103E000932F0100910901003073
:100A500089F00F3770F0F0DCB0918900A091880028
:100A600002E010E0A00FB11FB0938900A0938800AE
:100A700044C11AC0E6DC309189002091880030938F
:100A80002B0120932C01C1DDB0E0A5E043DDC6DCE5
:100A900033DC3CDC06E00093030108EE00932E01FA
:100AA00003E000932F0129C1C2DCB0918900A0911D
:100AB0008800A250B040B0938900A09388001DC167
:100AC00000910201013021F40027009302011895E2
:100AD00018950FEFA017B00711F0119618952196F1
:100AE000AA27BB27189500910101109100012091C0
:100AF0002F0130912E011317020769F0A89501E02C
:100B000005BDF0910101E09100013196F0930101E2
:100B1000E0930001189500E005BD00270093010156
:100B200000930001A8955B2F4A2F71E060E0A4DCE0
:100B30002F923F924F925F92DF93CF93CBDCCF9176
:100B4000DF914C2F5D2F31E0AFDC3F912F911F9152
:100B50000F919927400F511F621F731F891F06B500
:100B60001127222733279927400F511F621F731F18
:100B7000891FA89B0CC001E005BB002711E02227BC
:100B800033279927400F511F621F731F891F4093FE
:100B9000090150930A0160930B0170930C0180933B
:100BA0000D0140910D0130910C0120910B0110912C
:100BB0000A0100910901C2DC5093220160932301D4
:100BC000709324018093250190932601A093350111
:100BD0008CDB9CDB8ADB009103010630A1F00091E5
:100BE0002601A1DB009125019EDB009124019BDB06
:100BF0000091230198DB0091220195DB84DBF0E07A
:100C0000E2E3C0DB29C000913501003011F47BDB49
:100C100003C000913501AADB009126019ADB0CE2AA
:100C200079DB00912601A2DB009125017CDB0CE23F
:100C300071DB0091240177DB009123018ADB0EE256
:100C400069DB0091230192DB009122016CDB5BDB0D
:100C500008E460DB0AE75EDB3DDC06BD00930001D3
:100C60000093010100910301013031F40FEF0DBF3A
:100C700002E00EBFF894B7CD023031F40FEF0DBF94
:100C800002E00EBFF894E0CD033031F40FEF0DBF5A
:100C900002E00EBFF89412CE043031F40FEF0DBF16
:100CA00002E00EBFF89442CE053031F40FEF0DBFD5
:100CB00002E00EBFF89472CE063031F40FEF0DBF94
:100CC00002E00EBFF894B2CE1895FADA00DBF0E03D
:100CD000E2E258DB03DBF0E0EAE354DB06DBF0E0C2
:100CE000E0E550DB09DBF0E0E6E64CDBA895789424
:100CF000B3E0A4E80FDCE4DA0895FDDBFCDBEADB1B
:100D000001E00CBB01E00DBBA89578940000000049
:100D100000000000000000000000000000000000D3
:100D200000000000000000000000000000000000C3
:100D300000000000000000000000000000000000B3
:100D400000000000000000000000000000000000A3
:080FE00000000000000092CEA9
:00000001FF
